:100000001DC047C055C035C034C0B5C132C032C0B4
:1000100030C02FC02EC02DC02CC02BC02AC0010262
:100020000000040001020408102002020202020281
:1000300000000000380000000000370011241FBE3F
:10004000CFE5D2E0DEBFCDBF11E0A0E6B0E0E6E252
:10005000F6E002C005900D92A830B107D9F721E073
:10006000A8E0B1E001C01D92A531B207E1F7B1D21D
:10007000D8C2C6CF1F920F920FB60F9211248F9342
:1000800081E080930B018F910F900FBE0F901F9016
:1000900018951F920F920FB60F9211248F9381E043
:1000A000809309018F910F900FBE0F901F901895AC
:1000B0001F920F920FB60F9211248F939F93EF937D
:1000C000FF9380910A018F5F80930A0190910A014A
:1000D000E0910801F0E0E05AFF4F8081981730F07E
:1000E00010920A0198B380E1892788BBFF91EF91B4
:1000F0009F918F910F900FBE0F901F901895EF92C8
:10010000FF920F93CF93DF93C5E6D0E081EBE82E0B
:1001100080E0F82E29913991F701419151917F01A9
:10012000052E000C660B770B0AE084E043D068E2F2
:1001300070E080E090E09CD1F0E0C13BDF0751F738
:10014000F8948AE080BD88E088B993E094BB90E69B
:100150009BBF85BB82E085BF88E187BB84E088BB0D
:100160007894DF91CF910F91FF90EF900895809157
:100170000B01882349F0459B02C060E001C061E0AB
:1001800083E0DCD110920B0180910901882389F072
:1001900064E670E080E090E06BD1809108018430EB
:1001A00020F48F5F8093080102C010920801109222
:1001B000090108952F923F924F925F926F927F9222
:1001C0008F929F92AF92BF92CF92DF92EF92FF9267
:1001D0000F931F93CF93DF93CDB7DEB728970FB65A
:1001E000F894DEBF0FBECDBF382E4A015B01690116
:1001F000E12CF12C452B462B472B11F001111BC094
:10020000C701B60128960FB6F894DEBF0FBECDBF6A
:10021000DF91CF911F910F91FF90EF90DF90CF90E2
:10022000BF90AF909F908F907F906F905F904F9016
:100230003F902F901DC160E472E48FE090E0A50133
:100240009401CDD129013A010A3020F410E0015087
:10025000110902C009E010E0F801E350FF4F2081CE
:1002600030E040E050E0C301B201B9D1832D90E00D
:10027000FC01EC5DFF4F1491865D9F4FFC01649182
:10028000E62FF0E0EE0FFF1FE05DFF4F259034906A
:10029000FC018491E82FF0E0EE0FFF1FEA5CFF4FB6
:1002A000A591B4918C91812B8C932D833E834F83A8
:1002B0005887ABD069837A838B839C83012F009509
:1002C0002D813E814F815885421A530A2D833E83EA
:1002D0004F8358879AD0DC01CB0189809A80AB800C
:1002E000BC8088199909AA09BB092D813E814F81DB
:1002F00058858C159D05AE05BF05A8F4F1018081D8
:10030000812B8083C9012D833E834F835887D5D0AD
:10031000F101808180238083C201CFD058854F8135
:100320003E812D81D3CF28960FB6F894DEBF0FBE45
:10033000CDBFDF91CF911F910F91FF90EF90DF9094
:10034000CF90BF90AF909F908F907F906F905F9075
:100350004F903F902F90089580B7807F80BF80B7E7
:10036000806880BF8CB580648CBD8FEF8DBD80B7F9
:10037000876080BF08951F920F920FB60F921124CD
:100380002F933F938F939F93AF93BF9380910D01D2
:1003900090910E01A0910F01B091100130910C01CC
:1003A00026E0230F2D3730F029E8230F0396A11DF7
:1003B000B11D03C00296A11DB11D20930C018093B5
:1003C0000D0190930E01A0930F01B0931001809145
:1003D000110190911201A0911301B09114010196A5
:1003E000A11DB11D8093110190931201A0931301DF
:1003F000B0931401BF91AF919F918F913F912F9135
:100400000F900FBE0F901F9018952FB7F894609122
:100410000D0170910E0180910F01909110012FBF7D
:1004200008953FB7F8948091110190911201A09125
:100430001301B091140122B708B601FE05C02F3F89
:1004400019F00196A11DB11D3FBFBA2FA92F982FFA
:100450008827820F911DA11DB11DBC01CD0143E074
:10046000660F771F881F991F4A95D1F70895089541
:10047000CF92DF92EF92FF92CF93DF936B017C01DB
:10048000D0DFEB01C114D104E104F10479F0EFDF16
:10049000C8DF6C1B7D0B683E7340A0F381E0C81A77
:1004A000D108E108F108C851DC4FF2CFDF91CF91BC
:1004B000FF90EF90DF90CF9008958330910528F062
:1004C000880F991F04970197F1F708958AB5826004
:1004D0008ABD8AB581608ABD83B7887F836083BF08
:1004E000789489B7826089BF37DF86B1887786685C
:1004F00086B9379A0895813031F48AB58F778ABDED
:100500008AB58F7B07C0823039F48AB58F7D8ABD6A
:100510008AB58F7E8ABD0895833039F480B78F7D88
:1005200080BF80B78F7E80BF0895843031F48CB552
:100530008F7D8CBD8CB58F7E8CBD08950F931F93DE
:10054000CF93DF931F92CDB7DEB787FF11C08F77B0
:1005500041F0813041F0823041F0833041F08FEF43
:1005600007C085E005C082E003C084E001C083E0ED
:10057000282F30E0F901E25EFF4F8491F901EC5D34
:10058000FF4F1491F901E65DFF4F04910023D9F06C
:10059000882319F06983AFDF6981E02FF0E0EE0F67
:1005A000FF1FE05DFF4FA591B4918FB7611106C0A9
:1005B000F8949C91E12FE095E92303C0F894EC9125
:1005C000E12BEC938FBF0F90DF91CF911F910F9193
:1005D000089581B781BF7ADF92DDC9DDFECFA1E248
:1005E0001A2EAA1BBB1BFD010DC0AA1FBB1FEE1FAD
:1005F000FF1FA217B307E407F50720F0A21BB30BF8
:10060000E40BF50B661F771F881F991F1A9469F773
:1006100060957095809590959B01AC01BD01CF01CF
:060620000895F894FFCFDD
:100626000204080305F0005000500050005000502E
:100636000050007800280050005000500050005034
:100646000050007800280050005000500050005024
:100656000050007800280014001400140014001440
:100666000014001400140014001400140028006480
:1006760000000006010B0288014A010B0288014AAC
:1006860001000018012A029F015E012A029F015EF5
:1006960001000006010B0288014A010B0288014A8B
:1006A6000100004A015E0172010000720188019F8B
:1006B6000100009F01B801D20100000B02FFC8969D
:0806C6007D6457322116020089
:00000001FF
